:100000000C9446000C94D8010C94E5010C94650006
:100010000C9465000C9465000C9465000C946500CC
:100020000C9465000C9465000C9465000C946500BC
:100030000C9465000C9465000C9465000C949A0176
:100040000C9465000C9465000C9465000C9465009C
:100050000C94EF010C9465000C9465000C94650001
:100060000C9465000C9465000C9465000C9465007C
:100070000C9465000C9465000C9465000C9465006C
:100080000C9465000C9465000C94650011241FBE4F
:10009000CFEFD0E4DEBFCDBF11E0A0E0B1E0E2E100
:1000A000F5E000E00BBF02C007900D92A834B10745
:1000B000D9F721E0A8E4B1E001C01D92AE34B20747
:1000C000E1F70E941F020C9487020C94000010922A
:1000D000000110920101109202011092030110928E
:1000E0000401109205010895FC01E150FF4F808149
:1000F0008F5F808308954298E0E0F1E081918EBDAA
:100100000DB407FEFDCF81E0E630F807B9F7429A5B
:10011000089591ED980F9A3040F4DB01A050BF4F45
:10012000E82FF0E0E35FFE4F0BC090EA980F9A31A2
:1001300050F4DB01A050BF4FE82FF0E0EE53FF4F2B
:1001400080818C9308959FEB980F9A3140F4DB01E6
:10015000A050BF4FE82FF0E0EE51FF4FF1CF8032BB
:1001600029F4FB01E050FF4F108208958D3229F4ED
:10017000FB01E050FF4F80E2808308950F931F93AF
:10018000CF93DF938C01C0E0D0E0BE01F8018191F4
:100190008F010E9489002196C630D105B1F7DF9109
:1001A000CF911F910F910C947B009FE9980F99318B
:1001B00040F4DB01A050BF4FE82FF0E0EE53FF4FBB
:1001C0000BC09EEB980F993148F4DB01A050BF4F54
:1001D000E82FF0E0EE51FF4F80818C93089561503D
:1001E0007F4F835C9E4FFC018081FB0180830895DB
:1001F000089588E60E940401089581E08093B90083
:100200008BE48093B800089594EA9093BC00909199
:10021000BC0097FFFCCF9091B9008093BB0084E8AD
:100220008093BC008091BC0087FFFCCF8091B90017
:1002300088E98093BB0084E88093BC008091BC0077
:1002400087FFFCCF8091B90084E98093BC0080E0F7
:10025000089580E480937C00EAE7F0E08081836881
:100260008083089590917C00907F90937C00909182
:100270007C00982B90937C0080917A00806480931E
:100280007A0080917A0086FDFCCF209178008091E1
:10029000790090E0982F8827820F911D08951A9B6E
:1002A00005C0479A82B18C7F82B908954798119A08
:1002B000089586B1089582E081B983EA84B98CE912
:1002C00087B980EA8AB983E58CBD81E08DBD88B1AC
:1002D000887F88B9429A5D9A43988DB383608DBBBD
:1002E000E9E6F0E080818B608083E8E6F0E08081E1
:1002F0008460808380E88093B00083E88093B100BD
:10030000809106018093B30010928000E1E8F0E054
:1003100010828081856080838FEF90E090938900C8
:1003200080938800EFE6F0E080818162808378949A
:100330000C9467001F920F920FB60F9211248F93A7
:100340009F9385B192E0892785B986EE99EF9093C6
:100350008500809384008091480190914901019625
:1003600090934901809348010B97DCF0109249016A
:100370001092480180914A0190914B01019690930F
:100380004B0180934A0185B191E0892785B980911D
:100390004A0190914B01409724F010924B0110922A
:1003A0004A019F918F910F900FBE0F901F9018954B
:1003B0001F920F920FB60F9211248F9389B18F91D4
:1003C0000F900FBE0F901F9018951F920F920FB6AF
:1003D0000F9211240F900FBE0F901F9018951F922F
:1003E0000F920FB60F9211240F900FBE0F901F9017
:1003F00018958093B30008959093C5008093C4002E
:1004000088E08093C10086E08093C20008959091B7
:10041000C00095FFFCCF8093C6000895CF93DF9373
:10042000EC018991882319F00E940702FACFDF912D
:10043000CF9108950E94070280E090E00895CF9345
:10044000DF9300D000D000D0CDB7DEB70E945B01B3
:100450000E944F0186B1FE01319620E030E0E0902D
:100460004A01F0904B010091080110910901C90166
:100470008E0D9F1DB8010E945F02865F9E4FDC01BA
:100480008C9181932F5F3F4F803271F4C9018E0DA3
:100490009F1DB8010E945F02865F9E4FDC018C9118
:1004A000803211F4449A03C088B1807E88B9263026
:1004B0003105A9F6CE0101960E94BE00C9CF97FB77
:1004C000072E16F4009407D077FD09D00E9473021E
:1004D00007FC05D03EF4909581959F4F0895709547
:1004E00061957F4F0895AA1BBB1B51E107C0AA1F4E
:1004F000BB1FA617B70710F0A61BB70B881F991FC5
:100500005A95A9F780959095BC01CD010895F8946E
:02051000FFCF1B
:10051200E6E6E6E6E6E67D00160046526F686520EE
:1005220020576569686E61636874656E20202020BB
:10053200012000BEF4E0E6F8B8DCB40446BCD09E6C
:10054200A4E4BA3EA07CF0C4C4D6B676E6DE06EADF
:080552006E367CFC0EFE7E00FB
:00000001FF
